:020000040000FA
:1000000013022E006F00EF02030AEE02020A00083C
:10001000000C2600060010022600110225006500D3
:1000200040002600FF0C06000008FF0C060011022D
:10003000250000000602300065000008040C3100B5
:100040001E0C300008090009000C300008090009E6
:10005000100C300008090009000C300008090009E4
:100060006C048C050C02300008090009000C3000FB
:10007000080900091F0C300008090009000C3000B5
:1000800008090008FF0C330000090009070C0200F2
:10009000000C2500080C0500080C280069006A0007
:1000A0006B0070007200040C310008094000300041
:1000B000070C31000809060C31000809050C310055
:1000C0000809030C310008096B00000C3100150908
:1000D00010024307A80A010C31001509100243075A
:1000E000C60A020C310015091002F00E2D002D0376
:1000F0002D032D032D030D022C0010020F0E4307BC
:10010000DF0A2A046D00ED02830A8A068D0A400088
:100110003000040C310008098A056C07A50A650641
:10012000A50A0A06980A0A05010C21000A0C3200E9
:1001300001024307640AA102F202640A6A06640A21
:10014000900C33001E096A05640A6A040A04640AF2
:100150002B00900C8B0043062B0B110C0B06290077
:10016000140C2B062900170C4B0629001E0C6B06DD
:100170002900010C8B062800020CAB062800040C99
:10018000CB062800080CEB062800EC0A2B00120C0A
:100190000B062900150C2B062900180C4B0629000C
:1001A000100C6B062900100C8B062800200CAB06E7
:1001B0002800400CCB062800EB064A05EC0A2B0071
:1001C000130C0B062900160C2B062900190C4B06E4
:1001D00029001F0C6B0629002A06290B2A054A074D
:1001E000F60A900C33001E094A04290B0B020F0E6D
:1001F0004306290B6807020B09023000040C31008A
:100200000809290BC900070E300008070D0B070C61
:1002100031000809050C310008092807120B050CEC
:10022000310008094807170B070C31000809880737
:100230001F0B060C31000809030C31000809A80740
:10024000240B030C31000809C807290B060C3100E8
:1002500008098A04640AAA05FF0C3300740014021A
:100260003000050C31000809070C310008090E0C9C
:100270003000040C310008090009000C3000040CA7
:1002800031000809000900090009000914023000C2
:10029000030C31000809060C31000809290C300054
:1002A000040C310008090009000C3000040C310076
:1002B00008090009000900090009010C31001509AD
:1002C000900C90004306680BB402070C74012F0BCE
:1002D0000A0C2D00800C3300080C3000040C310097
:1002E00008090009000C3000040C3100080900095D
:1002F000080C3000040C310008090009000C300023
:10030000040C31000809ED026C0BAA0470007100A6
:100310004000420A280C430C290C470C570C360CA1
:0A032000420C570C580C2E0C020C76
:0203FE00420AB1
:00000001FF
